:020000020000FC
:041000000C940F0E2F
:04102C000C94920D81
:1010730012010002FF010020EB03F72F0000010221
:10108300030109021200010100803209040000007B
:10109300000000000C03410054004D0045004C00CB
:1010A3001C03410054003900300055005300420036
:1010B3003800320020004400460055000C03310084
:1010C3002E0030002E0035000403090413010C0127
:0810D30000000C000001701E7A
:1010DC0012BD01BDF89A00B50895F999FECF12BD65
:1010EC0001BD20BDFA9AF99A01E00895F999FECF55
:1010FC000C946E08F80104910895F801349131961E
:10110C002491890108950091610000930C0100E87D
:10111C000093610001E00093610005BF02E005BF90
:10112C000C94A708E3E6F0E000810E7F0083A895FD
:10113C0007EF04BFE0E6008108610083F08301E063
:10114C0008950E94890D0E94900DFDCF0895E8ED41
:10115C00F0E000810F771CD00068008341D009B506
:10116C0000FFFDCFE8EDF0E000810F7D11D00F7D89
:10117C000083E0EE00810E7F0BD00B7F0083E2EE4C
:10118C000081016005D00860008378940C94750B85
:10119C0000830081089500910D01002321F401E0EA
:1011AC0000930D01D4DFEDE1F2E00081018100FF3D
:1011BC000DC0008111811E7F1183008301E000931B
:1011CC00EA0000E00093EA0000931C0200E00093A8
:1011DC00E9000091E80003FF02C00E94F20B0895A1
:1011EC00A895E0E6F0E000810861008300E400834C
:1011FC00F1A3F0A3F5A3F4A301E006BBE1E80081A1
:10120C0003600083E2E6008104600083008103FF39
:10121C00FDCFF78FA89507EF04BFE0E600810861CA
:10122C000083F083E2E6008108600083F08322A152
:10123C0033A1F78FF68FF3A3F2A301E006BB2D3D8C
:10124C00354010F006E001C002E009BD08950E948F
:10125C002F0E239746D1F093090124D204811581D6
:10126C00012B51F43DD100910701002309F4C7C0B3
:10127C0000E000930701C3C0A9D102FFFDCF018597
:10128C0000930601018500930E01018500930F0167
:10129C0001850093100101850093110101850093D4
:1012AC00120100910A01209112013091110140911B
:1012BC00100150910F01109106011A9541F0125036
:1012CC00B9F01A95B9F11A9509F47DC096C0109130
:1012DC000E01113021F411E010930B0102C0F093B8
:1012EC000B0191D00C3F11F416D188C076D186C079
:1012FC008AD010910E01112329F01A9549F01A95F4
:10130C00A9F07CC0F0930B010C3F09F077C0ECCF37
:10131C0053D103C049D109F471C00D911C9141D135
:10132C000F3FC1F305E00093090168C011E0109371
:10133C000B01EACFD1D031F0025009F440C00A952C
:10134C0041F05CC0F8D00E94250F0FEF00930A010A
:10135C0055C0552319F05A9589F050C001E005BFCE
:10136C00F5BF0DEF04BF60D031D103FFFDCF5ED0D0
:10137C00F9BD58D008E000936000FFCF01E005BF35
:10138C00F5BF52D023D103FFFDCF50D04BD0F9BDC8
:10139C000FEF1FE004C009811A810150104009832E
:1013AC001A8309811A81012BB1F700E800936100BF
:1013BC0000910C01009361000C940000FFCF01E040
:1013CC0000930B011BC088D019F00A9541F016C090
:1013DC005350A0F4B0D002E0009308010FC050535A
:1013EC0039F05A9541F05F52A9F35A9599F306C01A
:1013FC0002E00883EFCF01E0FCCF9DD071D02396A3
:10140C00E4E00C943C0E50930101409300013093A6
:10141C0003012093020110811B7F108310811F7721
:10142C0010830895E8ED09C086D05AC071D058D009
:10143C00F894E0EECCD0016002C000810F770083FD
:10144C00089521974ED000910601035019F00250D7
:10145C00B9F00BC041D021F00A9559F00A9529F446
:10146C0000910A010C3F19F456D02196089567D0CB
:10147C00FCCF00910101018700910001018711C08F
:10148C0010910F0129D019F00A9571F0EECF1123AC
:10149C0029F01A9529F01A9519F003C005E0EECF42
:1014AC00F1871ED045D0E1CF105339F01A9539F0A1
:1014BC001F5271F01A9571F0F4CF08E5DFCF00E000
:1014CC0010E020E030E00E94930E0093F100E9CF91
:1014DC0002E0F6CF04E0F4CF00910E010023089552
:1014EC0022C00ED009D008D00093040109D000937B
:1014FC000501E8EEF0E00CC008830091F1000883D0
:10150C000091F1000895EBEE62D000620083E8EEEA
:10151C000081077F94CFF7DF02E00093080103E01E
:10152C0000930901089556D0008100FFFDCF089566
:10153C004DD002FFFDCF00810B7F00837ECF0E9438
:10154C002E0E3AD006C02DD00093F1002DD059F4B8
:10155C0041D0082F092BA9F039D002FD12C000810F
:10156C0000FFFDCF4424042D4394003289F30091F5
:10157C000B0100230D911C9131F311970E947C08F3
:10158C00E3CF24D000FFFDCF00810E7F00830081CC
:10159C0000FFFDCF008102FFFDCFCDDFE5E00C9415
:1015AC003B0E11970C9480080D911C910F5F1F4FEF
:1015BC001C930E930197089575D0828193810081BD
:1015CC001181801B910B0196DF010895E8EEF0E08C
:1015DC0000810895FBDF0E7F32CF0E942B0E62D06C
:1015EC0080819181A081B181AF71048115810052FC
:1015FC001040048315830AC000910B01002331F4C1
:10160C00A301920102E911E00E94BD0E4ED0D8F167
:10161C00662477242C0114C073DFF301EE56FE4FC1
:10162C00008301E0600E00E0701E01960091F20054
:10163C00002311F03AD0D8F4C9DF0B7F0083FDDE14
:10164C0034D0D0F2F301B096E238F040A8F6009115
:10165C00E80002FFFCCF0091F20024D024813581F8
:10166C00201B304024833583E1CF4ADFAA95AA237F
:10167C00E1F700910B01013079F62091F1008C011A
:10168C000E947308D2CF04811581012B21F09EDFBB
:10169C0002FFFDCF50DF9EDF008100FFFDCFE8E0B1
:1016AC000C94380EE0E0F1E00895FCDF0281138128
:1016BC00081719070895EBEEF0E0208121602083D4
:1016CC00018302810270012B0283EDEE0081026026
:1016DC000083EEEE0081000F00E0001F089500E093
:1016EC0009D000FD05C0F093E90010E302E0E3CF60
:1016FC0000E008950093E900EBEEF0E0008108951E
:10170C000F770132B9F5112379F11A9559F01A9521
:10171C0061F01A9569F01A9509F11A95D1F01A959C
:10172C00E9F026C00E942D0922C00E94270A1FC082
:10173C0026D000910901018701E00187F187F1872B
:10174C00009108010187F1870E94990A0E949E0A64
:10175C000EC015D000910801018707C002E000936C
:10176C00080100E0009309010AD00E94990A03C005
:10177C000E94890A02C001E0089500E00895E8EE95
:10178C00F0E00081077F0083089508950350F9F479
:10179C00112339F01A9551F01A9581F01A9599F098
:1017AC0016C004E016D00BEC10E103C011D007E911
:1017BC0010E1E6E1F2E000831183DDCF0CE109D00A
:1017CC0003EA10E1F6CF04D00FEB10E1F2CFD5CF46
:1017DC000CE000931902089528D100931B02D1D07C
:1017EC00212F112329F12A95E9F02250F1F02250F2
:1017FC0099F02A9549F0225061F02A9581F02A95AA
:10180C00E1F02A95E9F023C0003809F447C00C94A4
:10181C00860B0038E1F7C3C00023C9F71EC00023B4
:10182C00B1F72DC0033098F727C1033080F700C102
:10183C00003868F3033858F7C5C0013841F75DC16B
:10184C00013051F41AD0008100FD06C0FCCF0E947B
:10185C00860B002309F41ED008951091E300107834
:10186C00E4D00F77012B0093E30007D0008100FF39
:10187C00FDCFE3EE00810068C9C09FD0D1C081D0FC
:10188C00123040F49AD010931C02CAD000911C0262
:10189C000C94CB0BEBEEF0E07DD091C0BA93AA93F5
:1018AC00229700E0009318026CD0BFD0202F2A950D
:1018BC0019F02A95E9F022C002E10093190203E71E
:1018CC0010E1E6E1F2E000831183ADD00883ADD0E6
:1018DC00098373D00091190210E028813981021715
:1018EC001307A8F40F7181F401E0009318022EC0C5
:1018FC0002E10093190205E810E1E3CF0E94CC0B42
:10190C00002319F741D038C0F09318021FC0209360
:10191C0019021CC0008100FFFDCF10E0A6E1B2E06F
:10192C00012F1395003289F0ED91FC9111970491E0
:10193C000093F1002D913C912F5F3F4F3C932E93E0
:10194C00FD0103810A95038359F768D000911902B0
:10195C00002319F0008102FFDDCF2CD002FD0BC05B
:10196C0000911802013021F4008100FFFDCF58D006
:10197C00008102FFFDCF4CD000832296A991B99132
:10198C0008951091F1000895EBEEF0E003D0008182
:10199C00077F0895008100620083E8EE08950DD062
:1019AC0000911C02018706D00F770083008102FF93
:1019BC00FDCFA7C035D000810895E8EEF0E000819E
:1019CC00077F24C030D010911B02105829F01A95B3
:1019DC0019F01A9561F019C0F0DFF18700E000935F
:1019EC00F1001CD0008102FFFDCF12D00FC0E8EE39
:1019FC00F0E01081177F10830F7710E0F801E65E9E
:101A0C00FD4F00810093F100E9CFBEDF0083089504
:101A1C0000810B7F008300810F770895E8EEF0E0E2
:101A2C0000810E7FF3CF01D000D00091F10008951A
:101A3C0000911B02013039F00230E9F456D0D1F498
:101A4C00F4DF0F7719F44ED0A1DFE0CF0093E9005B
:101A5C0049D0108110FF0CC010811062108310E06F
:101A6C003ED021E0F801E65EFD4F208342D0EDCF61
:101A7C0036D0EACF0FDF089500911B02002311F03E
:101A8C00013019F42FD082DFC1CF023039F52DD0BF
:101A9C0021F52091F1002F772093E90023D00081CC
:101AAC0000FF19C079F000810061008301E010E0B3
:101ABC00422F0E94210E0093EA00F093EA0000816D
:101ACC000860008300E00BD030E0F901E65EFD4FCA
:101ADC0000830FD0D9CF03D0D6CFDCDE0895F0939E
:101AEC00E9000895EBEEF0E008959FDF4ADF002354
:101AFC00089563DF00810E7F0895BFDE008102FF31
:101B0C00FDCF86DF83CFE3E6F0E000810E7F00831C
:101B1C000C94AC080C94D1088A93FA93EA933A92F9
:101B2C002A921A920A927A936A935A934A933A9304
:101B3C002A931A930A938FB760D002FF05C05AD02C
:101B4C0002FF02C00BEF53D0E1EE008100FF0DC08D
:101B5C0051D000FF0AC00EEF4AD000810061008313
:101B6C000FEE45D04ED000623FD047D004FF0EC0E0
:101B7C0041D004FF0BC0E8ED00810F7D00830FEE18
:101B8C00018738D00F7E3CD000642ED036D005FFB4
:101B9C000DC030D005FF0AC000810F7E00830FED11
:101BAC0026D000810F7D2CD000681ED026D003FFDC
:101BBC000AC020D003FF07C007EF19D00E94750B95
:101BCC0020D0116011D08FBF0991199129913991B1
:101BDC00499159916991799109901990299039906D
:101BEC00E991F991899118951183008308950093D7
:101BFC00E1000895E2EE00810895E1EEF0E0FBCF04
:101C0C000083EDE1F2E000811181089500008895D8
:101C1C00FECF0EE50DBF02E00EBFCFEDD2E00E946D
:101C2C009808002311F00E94550E0E9489080E940A
:101C3C000C0E0C940C0E4A951AF0000F111FFBCFD2
:101C4C000895BA92AA929A928A927A926A925A9227
:101C5C004A92BA93AA939A938A930895BB84AA84BE
:101C6C00998488847F806E805D804C80BB81AA8142
:101C7C0099818881F0E00FB6F894CE0FDF1F0FBE6C
:101C8C00089520E006D0E9F70895259102D0E9F7F0
:101C9C0008952D9301501040202F212B08958FEC87
:101CAC0090E1FC0105911491FC013296A591B4913F
:101CBC00FC01349625913491422F432B19F0F901F4
:101CCC00E4DF01C0DEDF069610E18B3D910748F39F
:101CDC0008952F930CD02F9101D008953CD0F12F63
:101CEC00E02F45E047BFE89536D012D0089533D0A9
:101CFC00F12FE02F43E047BFE8952DD008952BD06E
:101D0C00F12FE02F43E047BFE89525D001D008958F
:101D1C0022D041E147BFE8951EC01DD0F12FE02F26
:101D2C0041E247BFC895002D16C015D0F12FE02F0A
:101D3C0049E047BFC895002D0EC0F32FE22F012EAE
:101D4C00102E41E047BFE89506C005D0002E29E0D3
:101D5C0027BFE89500C0022E27B720FDFCCF202D11
:101D6C000895022E27B726FDFCCF202D08950E9442
:101D7C00270E22974801C901DA0110C05BD001E09F
:101D8C00A00E00E0B01E00E4A01600E0B00608F4BF
:101D9C0040C0830120E030E00E94740E0A2F0B2B10
:101DAC0009F440C0082F0F7710E02C01401A510A9B
:101DBC00320100E4A02E03C00A2F0B2BE1F04816D1
:101DCC00590680F0F40101914F010983119729F014
:101DDC0001914F010883119711C0F20131960491C2
:101DEC0008830CC0F201049109833196E817F907B6
:101DFC00A1F7F401EDCF1BD0088319839201088160
:101E0C0019810E94A30E16D0AA94B1F62301AA241C
:101E1C00BB240DD0312F0F3F3F4F09F4AFCF8301BF
:101E2C001DD0B7CF01E02296ECE00C94340E820169
:101E3C000C94830802E0400E00E0501E08959A9323
:101E4C008A9380E090E08C0109D080589F4F8F3F9F
:101E5C000FE09007C0F389919991089520E030E04C
:101E6C000C947D0E00000000000000000000FC003F
:101FE4000C946F0E0C94930E0C949B0E0C94A30EF5
:0C1FF4000C94740E0C94850E0C94AB0E33
:0400000300001000E9
:00000001FF
